:0300000002383A89
:0C383A0078FFE4F6D8FD75816E0238813D
:100F080020000A3C2E2E2E3E004950436F6E6E651F
:100F180063745245510A004950436F6E6E6563749D
:100F2800000A49504E6F41434B210A003E432C565C
:100F38002C43432CC0E4E0EFF2E5F020D1E8EDEAE1
:100F4800EEEC49500A003E432C4D41432C253032EB
:100F580062583A25303262583A25303262583A257A
:100F6800303262583A25303262583A253032625867
:100F78002C4D414320E0E4F0E5F10A003E432C56B5
:100F880045522C20332E3220EEF220257320257373
:100F98002CC2E5F0F1E8FF20495020ECEEE4F3EB39
:100FA800FF0A004A616E2031342032303039003176
:100FB800313A32313A3334003E432C4C442C5052AF
:100FC8004F473A20202020202020202020202020A9
:100FD8002020202020202020202020202020202009
:100FE80020202020202020202020202020202020F9
:100FF80020202020202020202020202020202020E9
:1010080020202020202020202CC4E0F2E020EFF037
:10101800EEF8E8E2EAE828F4E0E9EB290A003E2ADB
:101028002C312CCEF1EDEEE2EDFBE520EFE0F0E027
:10103800ECE5F2F0FB20F1E5F2E5E2EEE3EE20E884
:10104800EDF2E5F0F4E5E9F1E00A003E412C41302B
:10105800312C2562752E2562752E2562752E256226
:10106800752C495020E0E4F0E5F120E0E4E0EFF2EF
:10107800E5F0E00A003E412C4130322C2562752E05
:101088002562752E2562752E2562752C495020E043
:10109800E4F0E5F120EEF1ED2E20F1E5F0E2E5F0E7
:1010A800E00A003E412C4130332C2562752E256222
:1010B800752E2562752E2562752C495020E0E4F0C6
:1010C800E5F120F0E5E72E20F1E5F0E2E5F0E00AB1
:1010D800003E412C4130342C2562752E2562752E38
:1010E8002562752E2562752CCCE0F1EAE020F1E549
:1010F800F2E80A003E412C4130352C2562752E2538
:1011080062752E2562752E2562752CD8EBFEE70ACE
:10111800003E2A2C312CC4EEEF2E20EFE0F0E0EC5C
:10112800E5F2F0FB20F1E5F2E5E2EEE3EE20E8ED92
:10113800F2E5F0F4E5E9F1E00A003E422C533031E3
:101148002C2562752CC6E4E0F2FC20E7E0EFF0EE17
:10115800F1E020F1EEE5E4E8EDE5EDE8FF20EEF260
:1011680020F1E5F0E2E5F0E00A003E422C5330328F
:101178002C2562752CCEE1ECE5ED20F120F1E5F0AF
:10118800E2E5F0EEEC20E1E5E720EAE2E8F2E0ED66
:10119800F6E8E90A003E422C5330332C2562752CC0
:1011A800CFE5F0E5E7E0EFF3F1EA20EFF0E820EF34
:1011B800EEF2E5F0E520F1E2FFE7E820F120F1E5C5
:1011C800F0E2E5F0EEEC0A003E422C5330352C25D7
:1011D80062752CCAE0EDE0EB20F8E8F0EEEAEEE20A
:1011E800E5F8E0F2E5EBFCEDEEE3EE20EEE1ECE510
:1011F800EDE00A003E532C5330362C25303262582D
:1012080025303262582530326258253032625825EE
:101218003032625825303262582C4D414320E0E488
:10122800F0E5F120F8E8F0EEEAEEE2E5F8E0F2E5C4
:10123800EBFCEDEEE3EE20EEE1ECE5EDE00A003E3E
:10124800454E440A000A44756D705820202020201D
:1012580030302030312030322030332030342030CC
:101268003520303620303720303820303920304192
:101278002030422030432030442030452030460082
:101288000A3A003A20000A000A44756D704420208A
:1012980020202030302030312030322030332030B0
:1012A800342030352030362030372030382030395F
:1012B8002030412030422030432030442030452027
:1012C800304600457272206B65790052642065656E
:1012D80070726F6D0A005264204D454D0A005264C9
:1012E80020436F64650A00577269746520436F6410
:1012F800650A0044656275674950204F4E0A0044EC
:10130800656275674950204F46460A004465627514
:101318006755736572204F6E0A004465627567559C
:10132800736572204F46460A0044656275674D73BF
:1013380067204F6E0A0044656275674D7367204FDA
:1013480046460A00436F6E666967206C6F636B21BF
:101358000A00577220656570726F6D0A002053612C
:10136800766520656570726F6D210A00457272207E
:101378004D414321004C6F61643E3E002A003C41D0
:1013880030313D003C4130323D003C4130333D007E
:101398003C4130343D003C4130353D003C21003C6F
:1013A8005330313D003C5330323D003C5330333DE7
:0D13B800003C5330353D003C5330363D00C5
:06434800010B0001090059
:10430B00C28E438910758BFF758DB7D2ABD28E22BF
:03001B000237AAFF
:1037AA00C0E0C083C082C0D0C28E758BFF758DB752
:1037BA0020060675A61E75A6E10509D202E50B606C
:1037CA0002050BE50AD394014002150A050EE50E1F
:1037DA00540F7048D20EE50E543F7012D200907A00
:1037EA00F5E0600A04F0E0D394B44002D206907A7D
:1037FA00F0E0600204F090756EE0600214F0907AD6
:10380A00F6E0D394014003E014F0300502050CE51C
:10381A000DD394644004D2068002050DE508D394C2
:10382A000140021508D28ED0D0D082D083D0E032A7
:10089B00C291C290D2B5C20B7D027C007F0712427F
:1008AB00D48F25E525646060097D017F6012426F5E
:1008BB00D20BE4FDFC7F0B1242D48F25E52530E6ED
:1008CB00097D04E4FF124293D20B7D017C007F076C
:1008DB001242D48F25E5257008FD7FFF12426FD29F
:1008EB000B300B03126000C288C2A8C2AA75890024
:1008FB00123BE69077A8E0B4FA06A3E064CE607BE7
:10090B00E4F52574A02525F582E43477F583E4F02E
:10091B000525E525B443EC9077A874FAF0A374CEC3
:10092B00F0A374CCF09077AE740AF0E4A3F0A304B8
:10093B00F0A3F09077A474FFF0A3F0A3F0E4A3F07E
:10094B009077BF740AF0E4F525E5252401FFE43325
:10095B00FE74A02525F582E43477F583E0FD124281
:10096B004B0525E525C3944340DFE4F5A775A61E8B
:10097B0075A6E1907FF0F0A3F080FE9077B374033F
:10098B00F0A374CCF0E49077B2F012358FC2B512AD
:10099B00323AC206123FBED20BC20DC20C9079E0A6
:1009AB007408F090771E7424F0E4A3F09077A8E01D
:1009BB00907720F09077A9E0907721F09077AAE0DC
:1009CB00907722F09077ABE0907723F09077ACE0C4
:1009DB00907724F09077ADE0907725F0750A01E4DD
:1009EB009079E1F0C207C208C209C20A1242242060
:1009FB000B19AF257E007D03123159E4FF123659D6
:100A0B007E0F7F08E4FBFDFC122E66907AF5E0600A
:100A1B00037401F0E490756EF0F50C9079DFF0F54E
:100A2B000D12430B75A70775A61E75A6E1D2AFE491
:100A3B00F50D90756EE07003121AE5907AF6E0648E
:100A4B0001701D9080007410F09080A874FFF0A3CB
:100A5B00F0A3F0A3F0E4907AF6F0D20BC20CC20D27
:100A6B00908008E0F52530E405D2077410F0E525F9
:100A7B0030E508D2099080087420F0E52530E608AF
:100A8B00D2089080087440F0E50CC3940340199091
:100A9B008002E4F0908001F0908000F0E50C940669
:100AAB004006E4F50C123FBE9080A0E07003123DAF
:100ABB00D49080B8E07003123CE19080D0E07003DA
:100ACB00123F62908000E07013300710122F6D9070
:100ADB00779BEFF0D394004003120026908002E046
:100AEB007006908000E06005D205020A3AC205E468
:100AFB00F50C90756EE06003020A3A200B129079A8
:100B0B00E2E0600C7E0F7F0A123071E49079E2F024
:100B1B00300912122B9A90779BEFF0D3940040057B
:100B2B00E0FF12431B200803020CB0122A1390772C
:100B3B009BEFF07003020A3A9077DFE054BF247FFB
:100B4B007003020C19147003020BF12402600302F0
:100B5B000C52200B077E0F7F11123071200F0302F6
:100B6B000CB09077B7E070069077BBE06067907A37
:100B7B00ECE0FF9077B7E0B50724907AEDE0FE90BC
:100B8B0077B8E0B50618907AEEE0FE9077B9E0B54D
:100B9B00060C907AEFE0FE9077BAE06E60379077B4
:100BAB00BBE06F6003020CB0907AEDE0FF9077BC76
:100BBB00E06F6003020CB0907AEEE0FF9077BDE03F
:100BCB006F6003020CB0907AEFE0FF9077BEE06F9E
:100BDB006003020CB0C2039079E17401F0120021A2
:100BEB00750A01020CB0907AF5E060037401F09085
:100BFB007AE4E0FF9077E1E06F6003020CB0907A4B
:100C0B00E4E004F0E4F50A9079DFF0020CB0300375
:100C1B0003020CB09077AEE07003020A3A9077BFF4
:100C2B00740AF012434FD203E4F50A9079DFF09087
:100C3B007AF004F0E4907AE3F0A3F0200B677E0FD8
:100C4B007F1F123071805E907AF5E060037401F0C3
:100C5B003003529077DFE020E74B9077E1E0FF9095
:100C6B007AE3E0FE6F600D907AEBE07007EE146FA5
:100C7B0070338013907AE3E004F090779BE0FFD31E
:100C8B00940440031240F190746A7482F0A37401CF
:100C9B00F09077E1E090746CF07E747F6A7D0312C4
:100CAB00394D020A3A200303020DC8E50A70681297
:100CBB00419BEF60237E787FDF9078E0E02404FD9A
:100CCB0012394D907AEBE070099077BFE0F50A028C
:100CDB000A3AE4F50A020A3A907AF0E0D3943C40DF
:100CEB0036907AEBE07030907AF004F0124335E4F2
:100CFB009078DFF0A37412F0907AE4E09078E1F052
:100D0B00A374FDF090756F63A2019078E363A20169
:100D1B007F1212258F809E12432A8F25E525B40161
:100D2B001590746A7483F0E4A3F07E747F6A7D027D
:100D3B0012394D020A3AE525D39401401C90746A8E
:100D4B007483F0A37401F0E52524FEA3F07E747F79
:100D5B006A7D0312394D020A3AE50A640160030207
:100D6B000A3A9079DFE004F0200B077E0F7F2912FF
:100D7B0030719077BFE0C394C85004E02432F090F8
:100D8B0079DFE0C39405400DC203E49079E1F012E2
:100D9B000021020A3A7C7A7DEC9077B3E0FAA3E06B
:100DAB00FB7F02123ADE7E787FDF9078E0E024044E
:100DBB00FD12394D9077BFE0F50A020A3AE50A6455
:100DCB00016003020A3A9079E1E014604624FE6068
:100DDB0042147003020EBB24046003020A3AE4F5CA
:100DEB000C200F139079E17404F09079DFE054013B
:100DFB00F0750A01020A3A9080027410F0E49079BF
:100E0B00E1F09079DF04F0750AFA907AEC74FFF058
:100E1B00020A3A907AECE07003020EA59078DF7428
:100E2B0080F09078E17401F0E4A3F0A304F0A374D4
:100E3B0030F0A3747BF0E4F52574E62525F582E408
:100E4B003478F583747DF074E72525F582E43478E6
:100E5B00F583E4F0E52524079078E0F07C7A7DECCF
:100E6B009077B3E0FAA3E0FB7F02123ADE7E787F45
:100E7B00DFE5252409FD12394D907AEBE0601B125A
:100E8B00434FD203E4F50A9079DFF0907AF004F047
:100E9B00E4907AE3F0A3F0020A3A300F07E490797A
:100EAB00E1F080069079E17404F0750AFA020A3ACF
:100EBB009080027410F0750A059079DFE06401FFF1
:100ECB00F09079E17401F0EF70199077BBE060134B
:100EDB00FCA3E0FDA3E0FEA3E0FF907AEC121F2839
:100EEB00020A3A9077B7E0FCA3E0FDA3E0FEA3E093
:0C0EFB00FF907AEC121F28020A3A80FED9
:010F070022C7
:100026009077E0E0B444047F0180027F009077DFA0
:10003600E0B447047E0180027E00EE5F604A90775E
:10004600A8E09077E1F09077A9E09077E2F09077DA
:10005600AAE09077E3F09077ABE09077E4F09077C2
:10006600ACE09077E5F09077ADE09077E6F09077AA
:10007600E07452F090771863A2019080A863A20101
:100086007F0612258F02089190779BE0C394085053
:100096000302089A9077A8E0FF9077E1E06F60038B
:1000A60002089A9077A9E0FF9077E2E06F6003027A
:1000B600089A9077AAE0FF9077E3E06F6003020862
:1000C6009A9077ABE0FF9077E4E06F600302089ABE
:1000D6009077ACE0FF9077E5E06F600302089A90B6
:1000E60077ADE0FF9077E6E06F600302089A9077BD
:1000F600E0E06444701A9080A8E0B4FF139077188B
:1001060063A2019080A863A2017F0612258F80104A
:1001160090771CE09080ACF090771DE09080ADF079
:10012600907AF5E060037401F0907AF67464F090CA
:1001360077E07452F09077DFE0646D600302029B13
:100146007BFF7A0F79341217EB7BFF7A0F794E908B
:1001560077A8E0F52EA3E0F52FA3E0F530A3E0F5B0
:1001660031A3E0F532A3E0F5331217EB752EFF75D8
:100176002F0F7530AB7531FF75320F7533B77BFFB7
:100186007A0F79841217EB7BFF7A0F79C01217EB7F
:100196007BFF7A1079261217EB7BFF7A1079539042
:1001A60077AEE0F52EA3E0F52FA3E0F530A3E0F55A
:1001B600311217EB7BFF7A10797D9077B7E0F52E39
:1001C600A3E0F52FA3E0F530A3E0F5311217EB7BA2
:1001D600FF7A1079AB9077BBE0F52EA3E0F52FA35D
:1001E600E0F530A3E0F5311217EB7BFF7A1079D9F1
:1001F6009077A4E0F52EA3E0F52FA3E0F530A3E079
:10020600F5311217EB7BFF7A1079FC9077A0E0F5B9
:100216002EA3E0F52FA3E0F530A3E0F5311217EB9E
:100226007BFF7A1179191217EB7BFF7A117942A2BB
:100236000FE433F52E1217EB7BFF7A117972907A61
:10024600EBE0F52E1217EB7BFF7A11799D907AF58C
:10025600E0F52E1217EB7BFF7A1179D0A201E43379
:10026600F52E1217EB7BFF7A1179FC907AE5E0F513
:100276002EA3E0F52FA3E0F530A3E0F531A3E0F5DA
:1002860032A3E0F5331217EB123C647BFF7A127946
:10029600471217EB229077DFE0644C70737E127F73
:1002A6004DFBFDFC122E669077E7E0F526A3E0F500
:1002B60027E4F529E5269077E9F0A3E527F07E12F5
:1002C6007F887C777DE97B02122E66E4F5288527F8
:1002D60082852683E0FF74E92528F582E43477F5E4
:1002E60083EFF00527E527700205260528E528B4E3
:1002F60010DC7E127F8B7C777DE97B10122E6605E3
:1003060029E529C3941040AC7E127F8E12307122EB
:100316009077DFE0646C7060F52A7E127F90FBFDBB
:10032600FC122E66E4F529E49077E9F0A3E52AF0BD
:100336007E127F887C777DE97B02122E66E4F528A3
:10034600A82AE6FF74E92528F582E43477F583EFD9
:10035600F0052A0528E528B410E67E127F8B7C7707
:100366007DE97B10122E660529E529C3940840B75E
:100376007E127F8E123071229077DFE0644B7061BF
:10038600F52874D12528F582E43477F583E06032C8
:1003960074D12528F582E43477F583E0F46023747C
:1003A600D12528F582E43477F583E0FF74E7252824
:1003B600F582E43477F583E0B507100528E528B41F
:1003C60008C090756E7432F00208919077DF742140
:1003D600F0300B030208917E127FCB1230710208B7
:1003E600919077DFE0B4521A200B077E127FD3126A
:1003F60030719077DF7472F07E777FDF7D08123878
:10040600C6229077DFE064497045200B077E127F95
:10041600DE1230719077E7E0F526A3E0F527E4F5E4
:1004260028852782852683E0FF74E92528F582E45E
:100436003477F583EFF00527E527700205260528B2
:10044600E528B480DC7E777FDF7D8A1238C622906D
:1004560077DFE064437046200B077E127FE612309A
:10046600719077E7E0F526A3E0F527E4F5288527E0
:1004760082852683E493FF74E92528F582E43477A0
:10048600F583EFF00527E527700205260528E52800
:10049600B480DB7E777FDF7D8A1238C6229077DFD5
:1004A600E0645A7053200B077E127FEF1230719072
:1004B60077E7E0F526A3E0F5277C777DE97B80AF3B
:1004C60027AE26124167E4F528852782852683E430
:1004D60093FF74E92528F582E43477F583EFF00578
:1004E60027E527700205260528E528B480DB7E77F8
:1004F6007FDF7D8A1238C6229077DFE0644460038E
:1005060002058F9077E7E0FF64447003020891EFDD
:10051600B4310CC20B7E127FFB123071020891902F
:1005260077E7E0B4300CD20B7E137F0712307102EE
:1005360008919077E7E0B4320CD20C7E137F141248
:1005460030710208919077E7E0B4330CC20C7E1349
:100556007F221230710208919077E7E0B4340CD212
:100566000D7E137F311230710208919077E7E0B467
:10057600350CC20D7E137F3E1230710208919077C2
:10058600E7E0FF12001E02089190756EE0701320DE
:100596000B077E137F4C1230719077DF7421F002C7
:1005A600089190756E7432F09077DFE0FFB45104D5
:1005B600C2AF80FEEF64577045200B077E137F5A4B
:1005C6001230719077E8E090779BF0E4F528907709
:1005D6009BE0FFE528C39F400302089174E92528A4
:1005E600F582E43477F583E0FF9077E7E025282469
:1005F60017F582E43476F583EFF0052880D09077FE
:10060600DFE0645360030206B2200B077E137F65AA
:100616001230719077A8E0FF907620E06F703C90E2
:1006260077A9E0FF907621E06F70309077AAE0FF1F
:10063600907622E0B507249077ABE0FF907623E032
:10064600B507189077ACE0FF907624E0B5070C90DC
:1006560077ADE0FF907625E06F60169077DF742126
:10066600F0300B030208917E137F7412307102087A
:1006760091E4F528E4F50DAF28FE74172528F582D8
:10068600E43476F583E0FD12424B0528E528C39451
:10069600FE40E1C2AFE4907FF0F0A3F0907FFD74DE
:1006A600AAF0A374FFF0A37455F080FE9077DFE004
:1006B600644F704C9077E7E0F526A3E0F527E52731
:1006C6004526700A200B077E137F7D123071200BA2
:1006D600077E137F84123071E4F52874E92528F526
:1006E60082E43477F583E0852782852683F0052723
:1006F600E527700205260528E528B480DE02089164
:100706009077DFE0FFB445219077E7E0FDA3E09026
:100716007FF0CDF0A3EDF0C2AF907FFD74AAF0A3F9
:1007260074FFF0A37455F080FEEF64656003020861
:100736009A9077E7E0FFA3E0907FF0CFF0A3EFF089
:10074600E4F526F527D3907FF1E09527907FF0E03A
:1007560095264020E4F50D2527FFE5263401FE8584
:100766002782852683E0FD12424B0527E527700286
:10077600052680D17E137F861239D4EF4E60201273
:1007860000039077AEEFF01200039077AFEFF01210
:1007960000039077B0EFF01200039077B1EFF07E90
:1007A600137F8C1239D4EF4E60201200039077B776
:1007B600EFF01200039077B8EFF01200039077B9CC
:1007C600EFF01200039077BAEFF07E137F921239A2
:1007D600D4EF4E60201200039077BBEFF0120003B7
:1007E6009077BCEFF01200039077BDEFF012000394
:1007F6009077BEEFF07E137F981239D4EF4E6020CB
:100806001200039077A4EFF01200039077A5EFF0A3
:100816001200039077A6EFF01200039077A7EFF08F
:100826007E137F9E1239D4EF4E602012000390771C
:10083600A0EFF01200039077A1EFF012000390777B
:10084600A2EFF01200039077A3EFF0E4F528E4F5A9
:100856000DE5282401FFE433FE74A02528F582E483
:100866003477F583E0FD12424B0528E528C394430F
:1008760040DCC2AFE4907FF0F0A3F0907FFD74AA55
:10088600F0A374FFF0A37455F080FE7E777FDF7DC2
:04089600081238C646
:01089A00223B
:10412F00AE07EEC39430400BEED394395005EE2416
:10413F00D0FF22EEC39461400BEED394665005EE90
:10414F0024A9FF22EEC39441400BEED394465005B1
:08415F00EE24C9FF22AF062285
:1042F100907717E004F07006907716E004F090775D
:0A43010016E0FEA3E0FF1242B7220F
:100003001242F112412FEFC454F0FEC0061242F126
:0800130012412FD0E02FFF2263
:103F0500E4907C4FF01242F1907C50EFF0C3943076
:103F15004018E0FFD394395011907C4FE0246FF5A1
:103F250082E43475F583EFF08011907C4FE0246FC7
:103F3500F582E43475F583E4F0800C907C4FE00461
:103F4500F0E0D3940840BE752D00752E00752F0046
:0C3F5500E4F5307B017A75796F12286F5B
:013F6100223D
:0439D4008E2B8F2C7B
:1039D800907716E4F0A374FFF01242F1EF606EF4F2
:1039E800606B852C82852B83E493B507EC752D01DC
:1039F800E52C252DF582E4352BF583E4936025909D
:103A08007717E0252DFF907716E03400FE1242B7B5
:103A1800E52C252DF582E4352BF583E493B50704D1
:103A2800052D80CCE52C252DF582E4352BF583E496
:103A38009370A6E52D24FFFFE434FFFE907717E08E
:103A48002FF0907716E03EF07E007F0122E4FEFF23
:013A5800224B
:10358F007E137FA41239D4EF4E70037F01227E1376
:10359F007FA71239D4EF4E600C1242F1EF24D024E2
:1035AF00FF920F8002D20F7E137FAD1239D4EF4EF0
:1035BF00600C1242F1EF24D0907AEBF08005E4908A
:1035CF007AEBF07E137FB31239D4EF4E600C1242B8
:1035DF00F1EF24D0907AF5F08005E4907AF5F07E43
:1035EF00137FB91239D4EF4E600C1242F1EF24D091
:1035FF0024FF92018002C2019077A863A201907A02
:10360F00E563A2017F0612258F30013B7E137FBF3A
:10361F001239D4EF4E6030120003907AE5EFF012BA
:10362F000003907AE6EFF0120003907AE7EFF012C2
:10363F000003907AE8EFF0120003907AE9EFF012AE
:0A364F000003907AEAEFF07F0022FA
:104063009079E0E0C3947C503D9079E0E0FE04F069
:10407300741E2EF582E43477F583EFF0BF0A2790A0
:1040830079E0E0FF04F0741E2FF582E43477F583C2
:10409300E4F09079E0E0FF123A599079E07408F087
:0740A30090771FE004F022FA
:103FBE009080007480F09077A063A201F583F58263
:103FCE0063A2017F0812258F9077A863A2019080CB
:103FDE008863A2017F0A12258F9080927407F0A346
:103FEE0074D0F0A37406F09077B2E0FF9080B1F039
:103FFE009080E1EFF09080957455F0A3F0908000E2
:0A400E007401F090800974F0F022B4
:103DD400908009E04410F09080A0E070609080A191
:103DE4007482F09080A874FFF0A3F0A3F0A3F07F96
:103DF400039080AEEFF0A374CBF09080007402F0D7
:103E0400907C43121F3400000000907C43E09080BB
:103E140040F0907C44E0908041F0907C45E09080BC
:103E240042F0907C46E0908043F0A3E4F0A3F0A33A
:0D3E3400F0A3F0908018F0A3F0A3F0A3F02D
:013E4100225E
:103F6200908009E04440F09080D17482F07F039009
:103F720080DEEFF0A374CCF09080027402F0907CAB
:103F820047121F3400000000907C47E0908058F0F8
:103F9200907C48E0908059F0907C49E090805AF003
:103FA200907C4AE090805BF0A3E4F0A3F0A3F0A33E
:0B3FB200F0908030F0A3F0A3F0A3F02B
:013FBD0022E1
:103CE100908009E04420F09080B8E0706C9080B939
:103CF1007482F07F039080C6EFF07FCDA3EFF07F59
:103D0100039080C4EFF0A374CDF09080C074FFF0F5
:103D1100A3F0A3F0A3F09080017402F0907C4B1209
:103D21001F3400000000907C4BE090804CF0907CB0
:103D31004CE090804DF0907C4DE090804EF0907C76
:103D41004EE090804FF0A3E4F0A3F0A3F0A3F09035
:093D51008024F0A3F0A3F0A3F01C
:013D5A002246
:103ADE008C268D27A907EAFDE975F018A424ACFF02
:103AEE00E5F034808F82F583EDF0EBFDE975F0188B
:103AFE00A4FFAEF024ACFBEE34808B82F583A3EDF5
:103B0E00F08527828C83E0FDEF24A8FFEE3480FE43
:103B1E008F82F583EDF08527828C83A3E08F828ED2
:103B2E0083A3F0852782852683A3A3E0FDE975F0A4
:103B3E0018A424A8FFE5F03480FE8F82F583A3A39A
:103B4E00EDF08527828C83A3A3A3E08F828E83A3BF
:043B5E00A3A3F0220B
:0638C6008D2BAB07AA06E2
:1038CC00908000E030E5079079E27401F022907C62
:1038DC0043E0FCA3E0FDA3E0FEA3E0F52F8E2E8DCC
:1038EC002D8C2CAE02AF038E838F8263A201E52E4A
:1038FC00540744C0F583852F8263A201AF2B122697
:10390C0001E4FCFDFEE52F252BF52FEE352EF52ED3
:10391C00ED352DF52DEC352CF52C908040E52CF06B
:10392C00A3E52DF0A3E52EF0A3E52FF09080007415
:10393C0020F0AF2FAE2EAD2DAC2C907C43121F2857
:01394C002258
:06394D008D26AB07AA065F
:10395300908002E030E5079079E27403F022907CD6
:1039630047E0FCA3E0FDA3E0FEA3E0F52A8E298D4A
:10397300288C27AE02AF038E838F8263A201E529D1
:10398300540744D0F583852A8263A201AF26122609
:1039930001E4FCFDFEE52A2526F52AEE3529F52965
:1039A300ED3528F528EC3527F527908058E527F0E5
:1039B300A3E528F0A3E529F0A3E52AF0908002749B
:1039C30020F0AF2AAE29AD28AC27907C47121F28E0
:0139D30022D1
:023659008F27B9
:10365B00908001E030E5099079E27402F07F00225E
:10366B00907C4BE0FCA3E0FDA3E0FEA3E0F52B8EEA
:10367B002A8D298C28907AE563A201E52A54074408
:10368B00C8F583852B8263A2017F06122617E52BD3
:10369B002406F52BE4352AF52AE43529F529E435FA
:1036AB0028F5289079E363A201E52A540744C8F56D
:1036BB0083852B8263A201AF27122617E4FCFDFE44
:1036CB00E52B2527F52BEE352AF52AED3529F5299E
:1036DB00EC3528F52890804CE528F0A3E529F0A3DC
:1036EB00E52AF0A3E52BF09080017420F0AF2BAE10
:0D36FB002AAD29AC28907C4B121F28AF2768
:01370800229E
:102F6D009081E0E0F5260526052605260526052691
:102F7D0005260526052605260526908010E0F5294F
:102F8D00A3E0F52AA3E0F52BA3E0F52C9081E1E079
:102F9D00F5260526052605260526052605260526DC
:102FAD00052605260526908014E0F52DA3E0F52EC7
:102FBD00A3E0F52FA3E0F530E52FB52B08E530B5EF
:102FCD002C037F0022E4F526E52F540744E0F5831A
:102FDD0085308263A2019077DF63A2017F081226FC
:102FED00479077E163A20190771863A2017F0612E3
:102FFD00258F9077DFE0F527A3E0F528E4F52690FF
:10300D0077DFE0702AA3E024F8F526E52F54074476
:10301D00E0F58385308274082582F582E43583F5E9
:10302D008363A2019077DF63A201AF26122647AE1C
:10303D0027E4FCFDE5302528F530E52F3EF52FED95
:10304D00352EF52EEC352DF52D908014E52DF0A3B4
:10305D00E52EF0A3E52FF0A3E530F090800074404D
:03306D00F0AF269B
:01307000223D
:102A13009081E6E0F52605260526052605260526EA
:102A230005260526052605260526908028E0F52996
:102A3300A3E0F52AA3E0F52BA3E0F52C9081E7E0D2
:102A4300F52605260526052605260526052605263B
:102A530005260526052690802CE0F52DA3E0F52E0E
:102A6300A3E0F52FA3E0F530E4F526E52FB52B0A17
:102A7300E530B52C05C208022B7FE52F540744F03F
:102A8300F58385308263A2019077DF63A2017F081B
:102A93001226479077DFE0F527A3E0F528E52845E0
:102AA3002770099080027410F07F0022907AECE086
:102AB300FFF460309077E1E06F6003022B46907A79
:102AC300EDE0FF9077E2E06F7079907AEEE0FF90AF
:102AD30077E3E06F706D907AEFE0FF9077E4E06F5B
:102AE3006031805F9077E1E0907AECF09077E2E0FC
:102AF300907AEDF09077E3E0907AEEF09077E4E06F
:102B0300907AEFF09077E5E0FFA3E09077B3CFF012
:102B1300A3EFF09077DFE0702AA3E024F8F526E531
:102B23002F540744F0F58385308274082582F5829B
:102B3300E43583F58363A2019077DF63A201AF26B7
:102B4300122647AE27E4FCFDE5302528F530E52FB6
:102B53003EF52FED352EF52EEC352DF52DAF2CAEA4
:102B63002BAD2AAC29AB30AA2FA92EA82DD3121F27
:102B73001740099080027410F07F002290802CE5AA
:102B83002DF0A3E52EF0A3E52FF0A3E530F0908020
:062B9300027440F0AF26C1
:012B99002219
:102B9A009081E3E0F5260526052605260526052665
:102BAA000526052605260526052690801CE0F5291A
:102BBA00A3E0F52AA3E0F52BA3E0F52C9081E4E04D
:102BCA00F5260526052605260526052605260526B3
:102BDA00052605260526908020E0F52DA3E0F52E92
:102BEA00A3E0F52FA3E0F530E4F526E52FB52B0A8F
:102BFA00E530B52C05C209022CF0E52F540744E84C
:102C0A00F58385308263A20190746E63A2017F0E00
:102C1A0012265D90746EE0F527A3E0F5289074768D
:102C2A00E0FFF4604A907AE5E0FEEF6E7079A3E087
:102C3A00FF907477E06F706F907AE7E0FF90747896
:102C4A00E06F7063907AE8E0FF907479E06F7057F4
:102C5A00907AE9E0FF90747AE06F704B907AEAE03C
:102C6A00FF90747BE06F703FE490747DF080089071
:102C7A00747D74FFF0D2D990746EE0702AA3E024B8
:102C8A00F2F526E52F540744E8F583853082740E61
:102C9A002582F582E43583F58363A20190746E631D
:102CAA00A201AF2612265DAE27E4FCFDE5302528F9
:102CBA00F530E52F3EF52FED352EF52EEC352DF5B9
:102CCA002DAF2CAE2BAD2AAC29AB30AA2FA92EA83A
:102CDA002DD3121F175006E5284527700990800149
:102CEA007410F07F0022908020E52DF0A3E52EF0ED
:102CFA00A3E52FF0A3E530F09080017440F0AF26F1
:012D0A0022A6
:043071008E2D8F2EE3
:10307500908000E030E5079079E27401F022907CC1
:1030850043E0FCA3E0FDA3E0FEA3E0F5348E338D21
:10309500328C31E534FFE5335407FEE42FF530EE8D
:1030A50034C0F52F853082F5837423F00530E53083
:1030B5007002052F532FC7F582852F83740AF005FB
:1030C50030E5307002052F532FC79077A863A20112
:1030D500852F8385308263A2017F0612260174063F
:1030E5002530F530E4352FF52F852D83852E826328
:1030F500A201852F8385308263A2011225E5E4FCB8
:10310500FDFE907C43E0F8A3E0F9A3E0FAA3E02FED
:10311500FFEE3AFEED39FDEC38FCEF2408FFE43E06
:10312500FEE43DFDE43CFC907C43121F28907C436B
:10313500E0908040F0907C44E0908041F0907C45A8
:10314500E0908042F0907C46E0908043F0908000D3
:033155007420F0F3
:013158002254
:0A2E66008E2B8F2C8C2D8D2E8B2FC0
:102E7000908000E030E5079079E27401F022907CC8
:102E800043E0FCA3E0FDA3E0FEA3E0F5358E348D26
:102E9000338C32E535FFE5345407FEE42FF531EE8F
:102EA00034C0F530853182F5837423F00531E53186
:102EB000700205305330C7F582853083740AF005FF
:102EC00031E531700205305330C79077A863A20115
:102ED00085308385318263A2017F06122601740644
:102EE0002531F531E43530F530852B83852C82632F
:102EF000A20185308385318263A2011225E58F36D8
:102F0000EF2531F531E43530F530E52F6017852DAB
:102F100083852E8263A20185308385318263A2017D
:102F2000AF2F122601E5362408252FF52FFFE4FCEC
:102F3000FDFEE5352FF535EE3534F534ED3533F559
:102F400033EC3532F532908040E532F0A3E533F0D2
:102F5000A3E534F0A3E535F09080007420F0AF35A0
:0C2F6000AE34AD33AC32907C43121F281D
:012F6C002242
:023A59008F3F9D
:103A5B00908000E030E5079079E27401F022907CD1
:103A6B0043E0FCA3E0FDA3E0FEA3E0F5438E428D13
:103A7B00418C40E543FFE5425407FEE42FFFEE3453
:103A8B00C090771E63A201F5838F8263A201AF3FC3
:103A9B00122601E4FCFDFEE543253FF543EE3542DE
:103AAB00F542ED3541F541EC3540F540908040E570
:103ABB0040F0A3E541F0A3E542F0A3E543F090808D
:103ACB00007420F0AF43AE42AD41AC40907C43124A
:023ADB001F28A2
:013ADD0022C6
:063159008E2A8F2BAB054E
:10315F00908000E030E5079079E27401F022907CD6
:10316F0043E0FCA3E0FDA3E0FEA3E0F5318E308D3C
:10317F002F8C2EE531FFE5305407FEE42FF52DEEB1
:10318F0034C0F52C852D82F5837423F0052DE52DA4
:10319F007002052C532CC7F582852C83EBF0052D7F
:1031AF00E52D7002052C9077A863A201852C8385ED
:1031BF002D8263A2017F061226017406252DF52D9F
:1031CF00E4352CF52C532CC7E52A852D82852C83CD
:1031DF00F0052DE52D7002052C532CC7F582852C9B
:1031EF0083E52BF0052DE52D7002052C532CC7E53B
:1031FF0031240AF531E43530F530E4352FF52FE47D
:10320F00352EF52E908040E52EF0A3E52FF0A3E5A7
:10321F0030F0A3E531F09080007420F0AF31AE3084
:0A322F00AD2FAC2E907C43121F2837
:013239002272
:1042B700A2AF9210C2AF438E2075D2028F828E8337
:0C42C700E0FFE4F5D2538EDFA21092AFAE
:0142D30022C8
:10424B00E5D220E0FBA2AF9210C2AF43D2028F8225
:10425B008E83EDF075D25063D250A21092AFE5D29F
:03426B0020E0FB55
:01426E00222D
:103BE600E4FDED2401FFE433FE1242B774A02DF587
:103BF60082E43477F583EFF00DBD3FE6E4FDED2476
:103C06007FFFE433FE1242B774972DF582E43475D4
:103C1600F583EFF074972DF582E43475F583E07043
:103C26001B74972DF582E43475F5837420F074982F
:103C36002DF582E43475F583E4F080040DBD80BE75
:103C4600E4907616F0FDEDFF7E001242B774172D54
:0D3C5600F582E43476F583EFF00DBDFEE954
:013C6300223E
:024167008B2BA0
:10416900A2AF9210C2AF85A22C53A2FE8E838F827A
:1041790005A28C838D82740912268BE52B53A2FE2E
:1041890043A22012268D53A2DF852CA2A21092AF42
:01419900FF26
:01419A002202
:1042D400A2AF9210C2AF8C838D82EF12268B43A2C1
:0C42E4002012268D53A2DFA21092AFFF23
:0142F00022AB
:02426F008F2698
:10427100A2AF9210C2AFE4F5838D82740612268B31
:10428100E52643A22012268D53A2DFA21092AF7F12
:01429100012B
:014292002209
:024293008F2674
:10429500A2AF9210C2AFE4F5838D82740A12268B09
:1042A500E52643A22012268D53A2DFA21092AF7FEE
:0142B5000107
:0142B60022E5
:1024B400A907E7FFA805EF93C3966008403B74FCA7
:1024C4002FFF80F00F08EF93C3966008402B74FB36
:1024D4002FFF80E00F08EF93C3966008401B74FA47
:1024E4002FFF80D00F08EF93D3966008400B74F948
:1024F4002FFF80C01F1F1F1F1FEF54FEF80303F799
:10250400E893FC08E893FD08E893FE08E893FF22AB
:1025140009E993C39D6008402974FB29F980F109F6
:10252400E993C39E6008401A74FA29F980E209E924
:1025340093D39F6008400B74F929F980D3191919B2
:102544001919E9C313C313FF22740093F8ECC39859
:102554004024701F740193F8EDC3984019701474EB
:0E2564000293F8EEC398400E7009740393F8CA
:10257200EFC39840037F00227F0122EDF8E6F008C6
:10258200A3DFFA22EDF8E0F608A3DFFA22E0A36364
:10259200A201F0A363A201DFF475A2002263A201EB
:1025A200F0A363A20122E0A363A201F0A363A2014C
:1025B200E0A363A201F0A363A201E463A201F0A37A
:1025C20063A201DFE175A20022E0A363A2016DFE16
:1025D200936CFDEE058393FC158363A201DFEA751C
:1025E200A200227F00E493A363A201F00F600CA378
:1025F200E583C2E3F58363A20180EA75A20022E0CB
:10260200A363A201F0A3E583C2E3F58363A201DF22
:10261200EE75A20022E0A363A201F0A3E583C2E467
:10262200D2E3F58363A201DFEC75A20022E0A3638B
:10263200A201F0A3E58344F8C2E5F58363A201DFBA
:10264200EC75A20022E583C2E3F583E0A363A20155
:10265200F0A363A201DFEE75A20022E583C2E4D2F9
:0A266200E3F583E0A363A201F0A3F7
:10266C0063A201DFEC75A20022E58344F8F583E058
:10267C00A363A201F0A363A201DFEE75A20022F90D
:10268C0022C002C004C00612FFF0D006D004D00253
:01269C00221B
:103709004572724C656E210A000A496E49503A00A9
:10371900205544502054696D654750530A00200ACA
:10372900495054696D653A2000200A444154414783
:1037390052414D3A20002049676E6F72650A200098
:103749002043414E2054696D654750530A00205467
:103759007261737353656E644552520A000ACEF85A
:10376900C4EBE8EDFB43414E210A000A4572724160
:10377900647243414E3A00205265496E6974204390
:10378900414E0A002043414E283029203E20544F03
:10379900210A0020545520300A0020545520310AAE
:0137A900001F
:03001E00E4FF22DA
:1041FC00C2A9438902758C48758A4875D90475DB48
:10420C004875DC4875DD4875DE48E4F5E9F5F9D20A
:08421C00D9C2DAD28CD2DE22F5
:1041CE00C2D9907B0BE07013E5E92419F5EB30D7DB
:1041DE0006E5F904F5FB2285F9FB22E5E924C8F58D
:0E41EE00EB30D706E5F904F5FB2285F9FB223C
:1040AA00C2D9907B0BE0702C301D16E5E92432F55D
:1040BA00EB30D707E5F904F5FB800385F9FBC21D50
:1040CA0022E5E92405F5EB30D706E5F904F5FB22EC
:1040DA0085F9FB22E5E92432F5EB30D706E5F90448
:0740EA00F5FB2285F9FB2222
:104224001241FC907B0BE0C394645006123B621273
:1042340041CE120022D21CE4F555907C23F0F544C3
:07424400F559C21DF55722D8
:1040F100EF24FCF544D3940D4010200B077E377F4D
:1041010009123071E4F544D21A229077E363A201D7
:10411100907C1363A201AF4412258FC21A200B0DAC
:0E4121007E377F127C777DE3AB44122E662240
:0F431B00D3EF6480948D5006E55970028F5922BC
:101AE50020D903021BE9201C03021BE9E5596067A5
:101AF50090746E540FFF7D46122586E5466401708D
:101B05003A90747DE0B4FF0ED21E200B127E377F13
:101B1500191230718009301E06E4F559021BE912CD
:101B250041CE123E42200B0D7E377F277C747D6EA1
:101B3500AB59122E66E4F559021BE91241CE123E4D
:101B450042200B0D7E377F327C747D6EAB59122E91
:101B550066E4F559021BE9E5446055907C17E024DD
:101B650005F526D3940D4007E4F544D21A80759007
:101B75007C13E526540FFF7D46122586E54630E7A2
:101B850002D21DE5466401701A301E17E549B401FD
:101B950012200B127E377F3F7C747D6EAB59122E5F
:101BA500668003123E421241CEE4F544D21A8034D7
:101BB500E556601E907AF7540FFF7D46122586E59F
:101BC50046B40103201E03123E421241CEE4F556EF
:101BD5008012201F0C907B0BE0C3946450031233DA
:101BE500171241CE122D0B8F26EF7003021D12E442
:101BF500F557E54630E70AE549B41905D2D9021D7E
:101C0500121240AAE546B4010CD21E200B077E37FE
:101C15007F49123071E558C394C8501B30031874BE
:101C25000C2558F582E4347BF583E5262558F558CF
:101C35007D46AF2612257D300121E54620E71C9023
:101C450079E37D46AF2612257DAF26123659EF7012
:101C55000A200B077E377F57123071E546548160A5
:101C650003021D12E526D3940D4010300B03021D0F
:101C7500127E377F66123071021D12E548D3940734
:101C8500401F300B03021D1290756F7D46AF261263
:101C9500257D7E377F747C757D6FAB26122E668021
:101CA5006CE50F30E662907C3EE0FF903ED393FEFC
:101CB500547F65467052EFA3936548704B907C3E08
:101CC500E0C313FF2425F582E4347CF583E0703806
:101CD500530F3F907C3EE0FD746F250FF582E43491
:101CE50061F583EEF0ED903ED493FE7470250FF50B
:101CF50082E43461F583EEF074252FF582E4347CBB
:101D0500F5837401F0430F40AF2612269D300E1A5D
:101D1500300015907B0BE0C39464500C0557E557D4
:101D250094F04004C2AF80FEC20E200203021E35AD
:101D3500906001E004F07006906000E004F0E55565
:101D45006031D39401400415558028907C23E0042C
:101D5500F0E0D39403400D200B077E377F801230CF
:101D650071124224200B077E377F8D123071E4F506
:101D750055D21C301B43E556703F907AF704F0A30B
:101D85007408F0A37480F0A37401F0A37406F090B6
:101D95007C0EE0907AFCF0907C0FE0907AFDF0905C
:101DA5007C10E0907AFEF0907C11E0907AFFF0E4F0
:101DB500A3F0A3F075560BC21B301972907C0CE092
:101DC5007035E5567031907AF77442F0A37408F0D7
:101DD500907C0DE0907AF9F0907C12E0907AFAF020
:101DE500A37401F0755606200B077E377F9C1230D1
:101DF50071907C0CE004F0907C0CE06402702FE59F
:101E050056702B907AF77402F0A37408F0907C0D4D
:101E1500E0907AF9F0A3F0A37401F0755606200B53
:101E2500077E377FA3123071907C0CE004F0C2026C
:051E35001220B8C200FC
:011E3A002285
:10419B00E558602CE49078DFF0A3E558F0907AE4D2
:1041AB00E09078E1F0A37419F0907B0C63A201907E
:1041BB0078E363A201AF5812258FE4F5587F0122F3
:0341CB007F002250
:0B432A00301A05C21A7F01227F00221A
:0100210022BC
:06434F00E4F558F54422DC
:0A433500E490756FF0A3F0A3F022EE
:103EA4002043616E457247495400200A00457272EE
:103EB4004C656E43616E21000A002043616E4572B9
:103EC40072434821000A205265714572722100C470
:103ED40000C401C402C403C404C405C406C407C89E
:103EE40000C801C802C803C804C805C806C807C278
:103EF40000C201C202C203C204C205C206C2070054
:013F040000BC
:102D0B00E59B541F6020200B1A7E3E7FA41230716E
:102D1B00E59B541FFF7E007D031231597E3E7FAE33
:102D2B00123071E4F59BE5BA30E010E4F5B375B100
:102D3B0080F5B2D21CF555907C23F0E5CFF47003EF
:102D4B00022E63752801E4F527E5CFF455287003AF
:102D5B00022E51E527C454F0F5B1E5B2547F64203F
:102D6B006003022E22E5B3540FF54A85BC46E5BD40
:102D7B00541FFF131313541FFFE5BD54E044184FAA
:102D8B00F547E5BDC43354E0FFE5BE131313541FE1
:102D9B004FF548E5BEC43354E0FFE5BF131313549E
:102DAB001F4FF54985A34B85A34C85A34D85A34E9A
:102DBB0085A34F85A35085A35185A352E4F5B2207B
:102DCB001F0FE546547EB5460843BDF875B35080DA
:102DDB000375B3D0E54A700AE546547EB546037FCA
:102DEB000022301F08E54630E7037F0022E54AD377
:102DFB009408401D200B177E3E7FB1123071AF4AF5
:102E0B007E007D031231597E3E7FBC1230717F00F4
:102E1B0022E54A2405FF22E5B2549F6023200B20B4
:102E2B007E3E7FBE123071AFB27E007D03123159F0
:102E3B00AFB37E007D031231597E3E7FBC123071E1
:102E4B00E4F5B275B3D0E52825E0F5280527E5278D
:0A2E5B00C394085003022D547F00B9
:012E6500224A
:103E4200907B0BE0C39464505675B180E4F5B3F5F2
:103E5200B28546BCE548C4135407FFE54754E04F1A
:103E6200F5BDE54833333354F8FFE549C41354072D
:103E72004FF5BEE54933333354F8F5BF854BA3857F
:103E82004CA3854DA3854EA3854FA38550A3855191
:103E9200A38552A3E54A540F2450F5B375550AC2BF
:023EA2001C22E0
:1033170075B190E5B220E613200B107E3E7FC912EF
:103327003071AFB27E007D03123159E4F5B3F5B2C7
:10333700E50F30E615E4F50F907C3EE02402F0E05F
:10334700903ED3937004907C3EF0746F250FF58206
:10335700E43461F583E0702D907C3EE0FFC31324D5
:1033670025F582E4347CF583E07005430F808015F2
:10337700E4F50F907C3EE02402F0E0903ED393709A
:1033870004907C3EF0E50F30E721907C3EE0FF9013
:103397003ED393F5BCE4F5BDEFA393FF333333542A
:1033A700F8F5BE75BF78430F408036746F250FF56B
:1033B70082E43461F583E0F5BC75BD807470250F38
:1033C700F582E43461F583E0FF33333354F8F5BE17
:1033D70075BF78050F050FE50FC394324003E4F579
:0533E7000F75B3502238
:09433F00EF6003C29622D296221F
:103B620043AB01C2E8C2EAE4FFEFC454F0F5B1C3CB
:103B7200EF64809488500575B3D08003E4F5B3E414
:103B8200F5B2F5BCF5BDF5BEF5BFF5C4F5C5F5C694
:103B9200F5C7F5A3F5A3F5A3F5A3F5A3F5A3F5A33F
:103BA200F5A30FBF0EC3907B0BE0FE25E0F5B475C5
:103BB200B50C75B66C75A11275AB0275C13E75C3B5
:103BC200FF75C203E4907C3EF0750F80FF7F199071
:103BD2007C25E4F0A3DFFCE4FF7F3290616FE4F028
:033BE200A3DFFC62
:013BE50022BD
:1013C5003E2A2C312CCFE0F0E0ECE5F2F0FB20F3E7
:1013D500EFF0E0E2EBFFFEF9E5E3EE20EAEEEDF2F9
:1013E500F0EEEBEBE5F0E020CACF20C8F1E5F2FC2A
:1013F5000A003E4C2C6B30312C25732C43EAEEF061
:10140500EEF1F2FC20EDE020F8E8EDE52043414E59
:101415002C30202D20353030EAE1283530EC292CD0
:1014250031202D203530EAE128353030EC290A000D
:1014350030202D20353030EAE1283530EC290031D7
:10144500202D203530EAE128353030EC29003E42A8
:101455002C6330312C2562752CC2F2EEF0E8F7EDE5
:10146500FBE920EAEEEDF2F0EEEBEBE5F020EDE046
:1014750020F8E8EDE50A003E2A2C312CCFE0F0E01B
:10148500ECE5F2F0FB20EFF0EEF2EEEAEEEBE02019
:10149500C8F1E5F2FC20EFEE20EFEEF0F2F320527A
:1014A500533233320A003E4C2C6B30352C256C758B
:1014B5002CD1EAEEF0EEF1F2FC20EEE1ECE5EDE008
:1014C50020EDE020EFEEF0F2F32C3130302C32300D
:1014D500302C3330302C3630302C313230302C3209
:1014E5003430302C343830302C393630302C3139DA
:1014F5003230302C33383430302C35373630302CD0
:101505003131353230300A003C21003C6B30313D01
:10151500003C6330313D003C6B30353D0043796321
:1015250054530A00537054530A0054550A00435447
:1015350049490A00435449540A0053705449540A0E
:101545000054696D655449540A000A4173796E6304
:101555004F55543A00CEF820E4EBE8EDFB210A00A4
:101565000A435243204552523A20000A4173796E8C
:1015750063494E3A00C4EBE8EDE03F3F3F0A003FC8
:101585003F3F0A000089129B24AD36BF48C15AD39C
:101595006CE57EF78108931AA52CB73EC940DB524E
:1015A500ED64FF76028B109926AF34BD4AC358D13E
:1015B5006EE77CF5830A9118A72EB53CCB42D9502E
:1015C500EF66FD74048D169F20A932BB4CC55ED70E
:1015D50068E17AF3850C971EA128B33ACD44DF560E
:1015E500E960FB72068F149D22AB30B94EC75CD5FE
:1015F5006AE378F1870E951CA32AB138CF46DD54EE
:10160500EB62F97008811A932CA53EB740C952DBED
:1016150064ED76FF89009B12AD24BF36C148D35ACD
:10162500E56CF77E0A8318912EA73CB542CB50D9BD
:1016350066EF74FD8B029910AF26BD34C34AD158AD
:10164500E76EF57C0C851E9728A13AB344CD56DF8D
:1016550060E972FB8D049F16A920BB32C54CD75E8D
:10166500E168F37A0E871C952AA338B146CF54DD7D
:1016750062EB70F98F069D14AB22B930C74ED55C6D
:10168500E36AF17800112332465765748C9DAFBE2D
:10169500CADBE9F810013322564775649C8DBFAE4D
:1016A500DACBF9E82130021367764455ADBC8E9F3D
:1016B500EBFAC8D93120120377665445BDAC9E8F2D
:1016C500FBEAD8C94253617004152736CEDFEDFC1D
:1016D5008899ABBA5243716014053726DECFFDEC0D
:1016E5009889BBAA6372405125340617EFFECCDDFD
:1016F500A9B88A9B7362504135241607FFEEDCCDED
:10170500B9A89A8B8495A7B6C2D3E1F008192B3AEC
:101715004E5F6D7C9485B7A6D2C3F1E018093B2ACC
:101725005E4F7D6CA5B48697E3F2C0D129380A1BBC
:101735006F7E4C5DB5A49687F3E2D0C139281A0BAC
:101745007F6E5C4DC6D7E5F48091A3B24A5B69789C
:101755000C1D2F3ED6C7F5E49081B3A25A4B79688C
:101765001C0D3F2EE7F6C4D5A1B082936B7A48597C
:101775002D3C0E1FF7E6D4C5B1A092837B6A58496C
:041785003D2C1E0FCA
:030023000233ECB9
:0D33EC00C0E0C0F0C083C082C0D075D01812
:1033F90030984AC298750B01AF9920200BEF6402EF
:10340900703BD220D2918035302207C222531F0F40
:10341900801CBF0904D2228024BF031285616B631B
:103429006180536180C220750B00C291800F741BAB
:103439002561F582E4346FF583EFF0056130996D0C
:10344900302168E568B4FF0C7599020568756C0050
:10345900D2908057E568B560077599030568804B78
:10346900E568D39560400DC221D224C290E4FF12D1
:10347900433F8037E56C6009F5990568756C0080F4
:103489002A741B2568F582E43470F583E0F56C64D1
:1034990002600BE56C64036005E56CB40905759978
:0D34A900098008856C990568756C00C29952
:0B34B600D0D0D082D083D0F0D0E03224
:103C64007BFF7A1379C51217EB907B0BE070147508
:103C74002EFF752F147530357BFF7A1379F71217E1
:103C8400EB8012752EFF752F147530447BFF7A1369
:103C940079F71217EB7BFF7A147953A21FE433F5FB
:103CA4002E1217EB7BFF7A14797C1217EB90746851
:103CB400E0FEA3E0FFC3E49FFFE49EFEAB07FAE44B
:103CC400F9F8FF7E8C7D0AFC121E778F318E308DC1
:0D3CD4002F8C2E7BFF7A1479AB1217EB2298
:1034C1007E157F0D1239D4EF4E70037F0122E490F7
:1034D1007B0BF07E157F101239D4EF4E601512422E
:1034E100F1BF3106907B0B740AF0BF3206907B0B63
:1034F1007464F07E157F161239D4EF4E600D123FC1
:1035010005EC4D4E4F24FF921F8002C21F7E157F96
:103511001C1239D4EF4E600D123F058F298E288D74
:10352100278C26800BE4752980752825F527F5263B
:10353100AB29AA28A927A8267F007E8C7D0A7C00BA
:10354100121E77121F09907468EEF0A3EFF0E47F6A
:10355100587E02FDFCAB29AA28A927A826D3121F51
:10356100175007756901D2238021E47F607E09FD30
:10357100FCAB29AA28A927A826D3121F1750077523
:0D3581006902C2238005756904C2237F0022
:01358E00221A
:10323A00E49061B2F09061A1F0906002F0C221C204
:10324A0024C220C222F568F560F508F561F50B90F5
:10325A00746874FFF0A374F4F09061037402F09040
:10326A00616CF090616EF0C21FE4907B0BF0C22398
:10327A001234C1E4F56A75F075E56AA42433F5825F
:10328A00E5F03468F583E4F0E56A75F00DA42404EA
:10329A00F582E43461F583E4F0F55F75F068E56A78
:1032AA00A42428F582E5F03471F58375F00DE55F05
:1032BA00121F65E4F0055FE55FB408DF056AE56A99
:1032CA00B408B3E4F56EF55AF55CF55DF567F56D8E
:1032DA00F55FF55BF56AF566C2ADF5C9D2CDD2CC1C
:1032EA00C2C9C2CAF5CDF5CC907468E0F5CBA3E0AB
:1032FA00F5CA85CBCD85CACCD29ED29CD2CAC2ACE5
:0D330A00C298C29975B81075B710D2AC22E8
:0100220022BB
:10269D008F2730230EE546B44209E54964027003E5
:1026AD0002286EE54754E324DF700302276224DF1E
:1026BD00700302274D14700302274D24E3700302AB
:1026CD00279714700302281914700302284A24E274
:1026DD0060282460600302286E300C077E157F226F
:1026ED00123071E54875F00DA42404F582E43461CF
:1026FD00F5837D46AF2712257D22E54875F00DA4A3
:10270D002404F582E43461F583E4F0300C077E1582
:10271D007F2912307175F00DE55DA424DBF582E59E
:10272D00F0346BF5837D46AF2712257D055D535D36
:10273D003FE55C655D600302286E055C535C3F22DE
:10274D00300C077E157F2F12307190711B7D46AFB7
:10275D002712257D22300C077E157F3312307175BF
:10276D00F00DE55AA424B3F582E5F03461F5837DCF
:10277D0046AF2712257D055A535A7FE55A656E607F
:10278D000302286E056E536E7F22300C077E157F77
:10279D003912307120234875F075E548A42440F5B1
:1027AD0082E5F03468F583E549541FFF1313543F58
:1027BD0075F00D121F657D46AF2712257D75F068EA
:1027CD00E548A42428F582E5F03471F583E54954F4
:1027DD001FFF1313543F75F00D121F65E4F02243D4
:1027ED00470143498075F068E548A42428F582E542
:1027FD00F03471F583E549543FFF1313543F75F0E1
:10280D000D121F657D467F0D12257D22300C077E32
:10281D00157F3F12307175F068E548A42428F582C4
:10282D00E5F03471F583E549543FFF1313543F75BB
:10283D00F00D121F657D467F0D12257D222023216F
:10284D00300C077E157F4612307175F075E548A482
:10285D002433F582E5F03468F5837D46AF271225E4
:02286D007D22CA
:103D5B008F2A90600363A20190701B63A201AF2AAC
:103D6B0012258FE4F562F563852A6590701B63A2BB
:103D7B000190158963A201AF65AE64AD63AC6212AD
:103D8B0025CB8F658E648D638C62741B252AF5821F
:103D9B00E43470F583E563F0741C252AF582E43472
:103DAB0070F583E562F0E52A2402F5607F0112438A
:103DBB003F7568FFD221D299200B0D7E157F4F7C6A
:093DCB00707D1BAB2A122E66224A
:104018008E2B8F2C8F828E83E5822404F582E435E3
:1040280083F583E02405F568D3940E400B200B2A12
:104038007E157F5A12307122852B83852C8263A2CC
:104048000174032566F582E43460F58363A201AF49
:0B4058006812258FE5682566F56622DA
:1022C500756602E4F52AE52AC3956940030224B33D
:1022D50090711BE0600D7E717F1B124018E49071B8
:1022E5001BF022E55D655C601B75F00DE55CA424C3
:1022F500DBF582E5F0346BAF82FE1240189061A1E8
:102305007406F022E4F568E55E1470030223C41434
:1023150070030223EC1470030224348000E4F55E9C
:102325003023030223BB75F075E56AA42433F582D7
:10233500E5F03468F583E06075E55B701875F07558
:10234500E56AA42433F582E5F03468AF82FE1240D5
:1023550018055B806175F075E56AA42436F582E59C
:10236500F03468F583E0540FFFE55BD39F50237588
:10237500F075E56AA42433F582E5F03468F58375D4
:10238500F00DE55B121F65AF82AE83124018055B49
:102395008024E4F55B75F075E56AA42433F582E5E0
:1023A500F03468F583E4F0056A536A078008E4F5BC
:1023B5005B056A536A07055EE56860030224AEE5BE
:1023C5005A656E601975F00DE56EA424B3F582E5C6
:1023D500F03461AF82FE124018056E536E7F055EC4
:1023E500E56860030224AEE56775F00DA42404F5E5
:1023F50082E43461F583E0602BE56775F00DA42474
:1024050004F582E43461AF82FE124018E56775F089
:102415000DA42404F582E43461F583E4F0056753E3
:10242500670780050567536707055EE568707A7578
:10243500F068E56DA42428F582E5F03471F583751F
:10244500F00DE55F121F65E0604C75F068E56DA461
:102455002428F582E5F03471F58375F00DE55F12FA
:102465001F65AF82AE8312401875F068E56DA42430
:1024750028F582E5F03471F58375F00DE55F121FDF
:1024850065E4F0055FE55FC39408401BE4F55F056F
:102495006D536D078011055FE55FC394084008E43F
:0E24A500F55F056D536D07055E052A0222CB1B
:0124B3002206
:1020B800E56775F00DA42404F582E43461F583E046
:1020C8007005056753670720231875F075E56AA43E
:1020D8002433F582E5F03468F583E07005056A532A
:1020E8006A0775F068E56DA42428F582E5F0347177
:1020F800F58375F00DE55F121F65E07011055FE56A
:102108005FC394084008E4F55F056D536D07300020
:102118002EC20090616DE004F09061B2E06002149C
:10212800F09061A1E0601814F0E07013906002E094
:1021380004F0E0D394034007E4F0055C535C3FE50A
:1021480008B40107E4F508D221D299E50BD39464C9
:102158004007C220E4F561F50B30210F90616DE076
:10216800D39414400BC221D2248005E490616DF011
:1021780020212BE50870279061A1E070211222C56B
:10218800E566D394024017E4906003F0A37419F055
:10219800AF66123D5BE4F566906000F0A3F0E56B76
:1021A80070030222C4F527E4F56BF562F563E527B1
:1021B800547FF565E5275480241BF582E4346FF5D8
:1021C8008363A20190158963A201AF65AE64AD6314
:1021D800AC621225CB8F658E648D638C62E52754C3
:1021E80080241BF582E4346FAF82F5288F295327AA
:1021F8007FE5634562601D300B030222C47E157FB4
:1022080065AB27AD29AC28122E667D03AF63AE629D
:1022180012315922200B0D7E157F70AB27AD29ACEA
:1022280028122E66852982852883A3E024E7600387
:102238000222BAE52724FCF556C3940E5066E556EB
:10224800C39404405F852982852883A3A3E0FF64A3
:10225800447020E5292407F582E43528F583E0B4A5
:1022680001119061A1E06007E4F0055C535C3FE474
:10227800F55622EFB44412E5292407F582E43528FF
:10228800F583E07004F55CF55DE5292402FFE4358B
:1022980028F5838F8263A201907AF763A201AF5673
:1022A80012258F22E4F556200B127E157F7A123004
:0C22B8007122200B077E157F841230710C
:0122C40022F7
:1038460002089BE493A3F8E493A34003F68001F2F5
:1038560008DFF48029E493A3F85407240CC8C33383
:10386600C4540F4420C8834004F456800146F6DF52
:10387600E4800B0102040810204080904348E47E57
:10388600019360BCA3FF543F30E509541FFEE49347
:10389600A360010ECF54C025E060A840B8E493A30E
:1038A600FAE493A3F8E493A3C8C582C8CAC583CA39
:1038B600F0A3C8C582C8CAC583CADFE9DEE780BEF1
:01434E00006E
:101E3B0075F008758200EF2FFFEE33FECD33CDCC5E
:101E4B0033CCC58233C5829BED9AEC99E5829840E1
:101E5B000CF582EE9BFEED9AFDEC99FC0FD5F0D6BE
:101E6B00E4CEFBE4CDFAE4CCF9A88222B800C1B9E8
:101E7B000059BA002DEC8BF084CFCECDFCE5F0CB26
:101E8B00F97818EF2FFFEE33FEED33FDEC33FCEB5F
:101E9B0033FB10D703994004EB99FB0FD8E5E4F91A
:101EAB00FA227818EF2FFFEE33FEED33FDEC33FC07
:101EBB00C933C910D7059BE99A4007EC9BFCE99AFB
:101ECB00F90FD8E0E4C9FAE4CCFB2275F010EF2F40
:101EDB00FFEE33FEED33FDCC33CCC833C810D70740
:101EEB009BEC9AE899400AED9BFDEC9AFCE899F87B
:0E1EFB000FD5F0DAE4CDFBE4CCFAE4C8F9220E
:0E1F0900C3E49FFFE49EFEE49DFDE49CFC22E9
:101F1700EB9FF5F0EA9E42F0E99D42F0E89C45F020
:011F27002297
:0C1F2800ECF0A3EDF0A3EEF0A3EFF0222C
:101F3400A8828583F0D083D082121F4B121F4B12CC
:101F44001F4B121F4BE473E493A3C583C5F0C583F1
:101F5400C8C582C8F0A3C583C5F0C583C8C582C8F7
:011F6400225A
:0C1F6500A42582F582E5F03583F5832287
:10178900E53A242EF8E6053A22782B301702782E0E
:10179900E475F001122018021F712010EB7F2ED280
:1017A900108018EF540F2490D43440D4FF30140B18
:1017B900EF24BFB41A0050032461FFE53B60021512
:1017C9003B053EE53E7002053D30170D782BE4756B
:1017D900F001122018EF021FB70240637403D217F9
:1017E9008003E4C217F53A8B2B8A2C892DE4F53B4B
:1017F900F53DF53EE53B60077F201217C480F5757E
:101809003CFFC211C210C212C213C215C216C218BD
:10181900121792FF700D3017057F001217D5AF3ED2
:10182900AE3D22B4255FC2D5C214121792FF24D04F
:10183900B40A00501A75F00A783B30D50508B6FF8E
:101849000106C6A426F620D5047002D21380D92435
:10185900CFB41A00EF5004C2E5D2140219D5D2113F
:1018690080C6D21080C0D21280BCD2D580BAD2151F
:1018790080B47F201217C42012077401B53B0040C1
:10188900F1121789FF1217C40217FDD218D2168058
:1018990095121789FB121789FA121789F94A4B70A1
:1018A9000679A67A1A7BFF20122EE53B602A7E0074
:1018B9008E82758300121F8A60060EEE653C70F0F9
:1018C900C2D5EBC0E0EAC0E0E9C0E0EE121A1CD0D4
:1018D900E0F9D0E0FAD0E0FB121F71FF60AAEBC07B
:1018E900E0EAC0E0E9C0E01217C4D0E02401F9D071
:1018F900E03400FAD0E0FBE53C0460DCD53CD9805B
:10190900877BFF7A1A7918D212809C791080027924
:1019190008C216C2188008D2D5790A8004790AC289
:10192900D5E53C047002F53CE4FAFDFEFF12178987
:10193900FC7B08201113121789FD7B1030100A1245
:101949001789FE121789FF7B20EC3382D592D55077
:1019590013C3E43010069FFFE49EFEE42011039DAB
:10196900FDE49CFCE4CBF8C211EC700CCFCECDCCDD
:10197900E824F8F870F38017C3EF33FFEE33FEED78
:1019890033FDEC33FCEB33FB994002FB0FD8E9EB59
:10199900301105F8D0E0C448B211C0E00AEC4D4E50
:1019A9004F78207B0070C2EAB53C0040BCC0E01211
:1019B9001A1ED0F0D0E0201104C4C0E0C4B211C096
:1019C900F01217ADD0F0D5F0EB0217FD1220771801
:1019D9009A53191458186B4C18674219184F192043
:0F19E90044192049188043192655190A46190A2E
:1019F80045190A471AC650186F2D18732E18962BBA
:101A08001877231894201AAF2A182F480000188E28
:101A18003F3F3F00790AA2D5201314301509B910A9
:101A2800020404B9080104A2D520160250010420BA
:101A380012689212B53B005034C0E07F2030131971
:101A48007F30A21272167215500F121A75C212C286
:101A580016C215C2187F30800F301503E9C0E01296
:101A680017C4301503D0E0F9D0E0B53BCC301517DA
:101A78007F30B9100C1217C47F583014077F788054
:101A880003B908031217C43012057F2D0217C47F4B
:101A9800202018F87F2B2016F322921280CF286E70
:101AA800756C6C2900D2111217893011F8C211789F
:101AB8003B30D50108F602182F2D5043495812170C
:101AC800892403B405004001E4901AC1931217B5A4
:0D1AD800743A1217B5D213753B04021914AD
:10286F008B2A8A2B892CE4F536F535F534F533F5BB
:10287F0031F532E52E452F452D6012EBC0E0EAC051
:10288F00E0E9C0E0AB2DAA2EA92F122028AB2A0514
:10289F002CE52CAA2B7002052B14F9121F71F5379A
:1028AF00C394094007E537D3940D40E1E537642021
:1028BF0060DBE537B42D054332038016E537B42BC3
:1028CF0005433201800C74FF252CF52C74FF352B3A
:1028DF00F52BE53060046410703FAB2AAA2BA92CAE
:1028EF00121F7164306009E530702E75300A80292F
:1028FF00900001121F8AFF64786004EFB4581343ED
:10290F0032017530107402252CF52CE4352BF52B84
:10291F008007E5307003753008AB2A052CE52CAA2B
:10292F002B7002052B14F9121F71F537C3946140F8
:10293F000AE537D3947A50035337DF74D02537F530
:10294F0037C3940A400CE5379411406D74F925375D
:10295F00F537E537D39530506043320185363B85E7
:10296F00353A853439853338AF307E00E4FCFDAB22
:10297F0036AA35A934A833121FC9C8ECC8C9EDC986
:10298F00CAEECACBEFCBE4FCFDFEEB2537F536EEF6
:10299F003AF535ED39F534EC38F533AF36AE35ADB4
:1029AF0034FCAB3BAA3AA939A838D3121F175003EE
:1029BF00022928433204022928E53220E003E4806B
:1029CF002DE52E452F452D601EAB2AE52C24FFF952
:1029DF00E52B34FFFAEBC0E0EAC0E0E9C0E0AB2D35
:1029EF00AA2EA92F122028E53230E20774FFFFFE2E
:1029FF00FDFC22E532AF36AE35AD34AC3330E103FA
:042A0F00021F092277
:101F7100BB010689828A83E0225002E722BBFE026E
:091F8100E32289828A83E49322A1
:101F8A00BB010CE58229F582E5833AF583E022500C
:101F9A0006E92582F8E622BBFE06E92582F8E22256
:0D1FAA00E58229F582E5833AF583E4932270
:101FB700BB010689828A83F0225002F722BBFE0109
:021FC700F32203
:101FC900E88FF0A4CC8BF0A42CFCE98EF0A42CFCB7
:101FD9008AF0EDA42CFCEA8EF0A4CDA8F08BF0A435
:101FE9002DCC3825F0FDE98FF0A42CCD35F0FCEB94
:101FF9008EF0A4FEA9F0EB8FF0A4CFC5F02ECD3959
:0F200900FEE43CFCEAA42DCE35F0FDE43CFC22C5
:10201800FAE6FB0808E6F925F0F618E6CA3AF622C9
:10202800BB011A89828A83D0F0D0E0F8D0E0F9D0D9
:10203800E0FAD0E0FBE8C0E0C0F00220A65016E9C4
:10204800F8D083D082D0E0F9D0E0FAD0E0FBC082AB
:10205800C08302209DBBFE16E9F8D083D082D0E071
:0F206800F9D0E0FAD0E0FBC082C0830220AF22A3
:10207700D083D082F8E4937012740193700DA3A3F8
:1020870093F8740193F5828883E47374029368600C
:06209700EFA3A3A380DF0C
:09209D00EBF608EAF608E9F62268
:0920A600EBF0A3EAF0A3E9F0223B
:0920AF00EBF208EAF208E9F22262
:00000001FF
